LX51 LINKER/LOCATER V4.66.1.0                                                           07/21/2017  11:34:04  PAGE 1


LX51 LINKER/LOCATER V4.66.1.0, INVOKED BY:
D:\KEIL\C51\BIN\LX51.EXE ..\Library\FU68xx_Hardware_Driver\Source\FU68xx_CFG.LIB, ..\Library\FU68xx_Hardware_Driver\Sour
>> ce\FU68xx_Flash.LIB, ..\Library\FU68xx_Hardware_Driver\Source\FU68xx_OSC.LIB, ..\Library\FU68xx_Hardware_Driver\Sourc
>> e\FU68xx_Power.LIB, ..\Library\FU68xx_Hardware_Driver\Source\FU68xx_WDT.LIB, .\Output\main.obj, .\Output\Interrupt.ob
>> j, .\Output\UARTInit.obj TO .\Output\FU68xx_UART_Demo PRINT (.\Listing\FU68xx_UART_Demo.map) REMOVEUNUSED


CPU MODE:     8051 MODE
MEMORY MODEL: LARGE


INPUT MODULES INCLUDED:
  .\Output\main.obj (MAIN)
         COMMENT TYPE 0: C51 V9.52.0.0
  .\Output\Interrupt.obj (INTERRUPT)
         COMMENT TYPE 0: C51 V9.52.0.0
  .\Output\UARTInit.obj (UARTINIT)
         COMMENT TYPE 0: C51 V9.52.0.0
  D:\KEIL\C51\LIB\C51L.LIB (?C_STARTUP)
         COMMENT TYPE 1: A51 / ASM51 Assembler
  D:\KEIL\C51\LIB\C51L.LIB (?C?CLDPTR)
         COMMENT TYPE 1: A51 / ASM51 Assembler
  D:\KEIL\C51\LIB\C51L.LIB (?C?ILDIX)
         COMMENT TYPE 1: A51 / ASM51 Assembler
  D:\KEIL\C51\LIB\C51L.LIB (?C_INIT)
         COMMENT TYPE 1: A51 / ASM51 Assembler


ACTIVE MEMORY CLASSES OF MODULE:  .\Output\FU68xx_UART_Demo (MAIN)

BASE        START       END         USED      MEMORY CLASS
==========================================================
C:000000H   C:000000H   C:00FFFFH   00014CH   CODE
X:000000H   X:000000H   X:00FFFFH   000001H   XDATA
I:000000H   I:000000H   I:0000FFH   000001H   IDATA
I:000000H   I:000000H   I:00007FH   000008H   DATA


MEMORY MAP OF MODULE:  .\Output\FU68xx_UART_Demo (MAIN)


START     STOP      LENGTH    ALIGN  RELOC    MEMORY CLASS   SEGMENT NAME
=========================================================================

* * * * * * * * * * *   D A T A   M E M O R Y   * * * * * * * * * * * * *
000000H   000007H   000008H   ---    AT..     DATA           "REG BANK 0"
000008H   000008H   000001H   BYTE   UNIT     IDATA          ?STACK

* * * * * * * * * * *   C O D E   M E M O R Y   * * * * * * * * * * * * *
000000H   000002H   000003H   ---    OFFS..   CODE           ?CO??C_STARTUP?0
000003H   00004FH   00004DH   BYTE   UNIT     CODE           ?PR?UART_ISR?INTERRUPT
000050H   00005AH   00000BH   BYTE   UNIT     CODE           ?PR?MAIN?MAIN
00005BH   000062H   000008H   BYTE   UNIT     CODE           ?PR?_UART_SENDDATA?UARTINIT
000063H   000065H   000003H   BYTE   OFFS..   CODE           ?INTERRUPT?00063
000066H   0000F1H   00008CH   BYTE   UNIT     CODE           ?C_C51STARTUP
0000F2H   000120H   00002FH   BYTE   UNIT     CODE           ?C?LIB_CODE
000121H   000144H   000024H   BYTE   UNIT     CODE           ?PR?UART_INIT?UARTINIT
000145H   000149H   000005H   BYTE   UNIT     CODE           ?C_INITSEG
00014AH   00014AH   000001H   BYTE   UNIT     CODE           ?PR?SOFTWAREINIT?MAIN
00014BH   00014BH   000001H   BYTE   UNIT     CODE           ?PR?HARDWAREINIT?MAIN

* * * * * * * * * * *  X D A T A   M E M O R Y  * * * * * * * * * * * * *
000000H   000000H   000001H   BYTE   UNIT     XDATA          ?XD?INTERRUPT

* * * * * * * * *   R E M O V E D     S E G M E N T S   * * * * * * * *
   *DEL*:           000033H   BYTE   UNIT     CODE           ?PR?_UART_SENDSTRING?UARTINIT
LX51 LINKER/LOCATER V4.66.1.0                                                         07/21/2017  11:34:04  PAGE 2


   *DEL*:           000003H   BYTE   UNIT     XDATA          ?XD?_UART_SENDSTRING?UARTINIT



OVERLAY MAP OF MODULE:   .\Output\FU68xx_UART_Demo (MAIN)


FUNCTION/MODULE                 BIT_GROUP   DATA_GROUP 
--> CALLED FUNCTION/MODULE     START  STOP  START  STOP
=======================================================
UART_ISR/INTERRUPT             ----- -----  ----- -----
  +--> _UART_SENDDATA/UARTINIT

_UART_SENDDATA/UARTINIT        ----- -----  ----- -----

*** NEW ROOT *****************

?C_C51STARTUP                  ----- -----  ----- -----
  +--> MAIN/MAIN
  +--> ?C_INITSEG

MAIN/MAIN                      ----- -----  ----- -----
  +--> UART_INIT/UARTINIT
  +--> SOFTWAREINIT/MAIN
  +--> HARDWAREINIT/MAIN

UART_INIT/UARTINIT             ----- -----  ----- -----

SOFTWAREINIT/MAIN              ----- -----  ----- -----

HARDWAREINIT/MAIN              ----- -----  ----- -----

?C_INITSEG                     ----- -----  ----- -----



PUBLIC SYMBOLS OF MODULE:  .\Output\FU68xx_UART_Demo (MAIN)


      VALUE       CLASS    TYPE      PUBLIC SYMBOL NAME
      =================================================
      010000F2H   CODE     ---       ?C?CLDPTR
      00000000H   NUMBER   ---       ?C?CODESEG
      0100010BH   CODE     ---       ?C?ILDIX
      00000000H   NUMBER   ---       ?C?XDATASEG
      010000ADH   CODE     ---       ?C_START
      01000000H   CODE     ---       ?C_STARTUP
      0100005BH   CODE     ---       _UART_SendData
*DEL*:00000000H   CODE     ---       _UART_SendString
*SFR* 000000D0H.6 DATA     BIT       AC
*SFR* 000000E0H   DATA     BYTE      ACC
*SFR* 000000F0H   DATA     BYTE      B
*SFR* 00000086H   DATA     BYTE      CFGKEY
*SFR* 000000D5H   DATA     BYTE      CMP_CR0
*SFR* 000000D6H   DATA     BYTE      CMP_CR1
*SFR* 000000DAH   DATA     BYTE      CMP_CR2
*SFR* 000000D7H   DATA     BYTE      CMP_SR
*SFR* 000000D0H.7 DATA     BIT       CY
*SFR* 00000082H   DATA     WORD      DP
*SFR* 00000083H   DATA     BYTE      DPH
*SFR* 00000082H   DATA     BYTE      DPL
*SFR* 000000F8H   DATA     BYTE      DRV_OUT
*SFR* 000000A8H.7 DATA     BIT       EA
*SFR* 000000A8H.4 DATA     BIT       ES0
*SFR* 000000D9H   DATA     BYTE      EVT_FILT
LX51 LINKER/LOCATER V4.66.1.0                                                         07/21/2017  11:34:04  PAGE 3


*SFR* 000000A8H   DATA     BIT       EX0
*SFR* 000000A8H.2 DATA     BIT       EX1
*SFR* 000000D0H.5 DATA     BIT       F0
*SFR* 000000D0H.1 DATA     BIT       F1
*SFR* 00000084H   DATA     BYTE      FLKEY
*SFR* 000000E8H   DATA     BYTE      FOC_SET0
*SFR* 000000E9H   DATA     BYTE      FOC_SET1
*SFR* 000000E8H.7 DATA     BIT       FOCEN
*SFR* 00000080H   DATA     BIT       GP00
*SFR* 00000080H.1 DATA     BIT       GP01
*SFR* 00000080H.2 DATA     BIT       GP02
*SFR* 00000080H.3 DATA     BIT       GP03
*SFR* 00000080H.4 DATA     BIT       GP04
*SFR* 00000080H.5 DATA     BIT       GP05
*SFR* 00000080H.6 DATA     BIT       GP06
*SFR* 00000080H.7 DATA     BIT       GP07
*SFR* 00000090H   DATA     BIT       GP10
*SFR* 00000090H.1 DATA     BIT       GP11
*SFR* 00000090H.2 DATA     BIT       GP12
*SFR* 00000090H.3 DATA     BIT       GP13
*SFR* 00000090H.4 DATA     BIT       GP14
*SFR* 00000090H.5 DATA     BIT       GP15
*SFR* 00000090H.6 DATA     BIT       GP16
*SFR* 00000090H.7 DATA     BIT       GP17
*SFR* 000000A0H   DATA     BIT       GP20
*SFR* 000000A0H.1 DATA     BIT       GP21
*SFR* 000000A0H.2 DATA     BIT       GP22
*SFR* 000000A0H.3 DATA     BIT       GP23
*SFR* 000000A0H.4 DATA     BIT       GP24
*SFR* 000000A0H.5 DATA     BIT       GP25
*SFR* 000000A0H.6 DATA     BIT       GP26
*SFR* 000000A0H.7 DATA     BIT       GP27
*SFR* 000000B0H   DATA     BIT       GP30
*SFR* 000000B0H.1 DATA     BIT       GP31
*SFR* 000000B0H.2 DATA     BIT       GP32
*SFR* 000000B0H.3 DATA     BIT       GP33
*SFR* 000000B0H.4 DATA     BIT       GP34
*SFR* 000000B0H.5 DATA     BIT       GP35
*SFR* 000000B0H.6 DATA     BIT       GP36
*SFR* 000000B0H.7 DATA     BIT       GP37
      0100014BH   CODE     ---       HardwareInit
*SFR* 000000A8H   DATA     BYTE      IE
*SFR* 00000088H.2 DATA     BIT       IF0
*SFR* 000000B8H   DATA     BYTE      IP0
*SFR* 000000C0H   DATA     BYTE      IP1
*SFR* 000000C8H   DATA     BYTE      IP2
*SFR* 000000D8H   DATA     BYTE      IP3
*SFR* 00000088H   DATA     BIT       IT00
*SFR* 00000088H.1 DATA     BIT       IT01
*SFR* 00000088H.3 DATA     BIT       IT10
*SFR* 00000088H.4 DATA     BIT       IT11
*SFR* 000000DCH   DATA     WORD      LPF_K
*SFR* 000000DDH   DATA     BYTE      LPF_KH
*SFR* 000000DCH   DATA     BYTE      LPF_KL
*SFR* 000000DEH   DATA     WORD      LPF_X
*SFR* 000000DFH   DATA     BYTE      LPF_XH
*SFR* 000000DEH   DATA     BYTE      LPF_XL
*SFR* 000000E6H   DATA     WORD      LPF_Y
*SFR* 000000E7H   DATA     BYTE      LPF_YH
*SFR* 000000E6H   DATA     BYTE      LPF_YL
*SFR* 000000DBH   DATA     BYTE      LVSR
      01000050H   CODE     ---       main
*SFR* 000000A8H.5 DATA     BIT       MCDIE
*SFR* 00000088H.6 DATA     BIT       MCDIF
*SFR* 000000C4H   DATA     BYTE      MD_DA0
LX51 LINKER/LOCATER V4.66.1.0                                                         07/21/2017  11:34:04  PAGE 4


*SFR* 000000C5H   DATA     BYTE      MD_DA1
*SFR* 000000C6H   DATA     BYTE      MD_DA2
*SFR* 000000C7H   DATA     BYTE      MD_DA3
*SFR* 000000C6H   DATA     WORD      MD_DAH
*SFR* 000000C4H   DATA     WORD      MD_DAL
*SFR* 000000CCH   DATA     BYTE      MD_DB0
*SFR* 000000CDH   DATA     BYTE      MD_DB1
*SFR* 000000CEH   DATA     BYTE      MD_DB2
*SFR* 000000CFH   DATA     BYTE      MD_DB3
*SFR* 000000CEH   DATA     WORD      MD_DBH
*SFR* 000000CCH   DATA     WORD      MD_DBL
*SFR* 000000C2H   DATA     WORD      MD_MA
*SFR* 000000C3H   DATA     BYTE      MD_MAH
*SFR* 000000C2H   DATA     BYTE      MD_MAL
*SFR* 000000CAH   DATA     WORD      MD_MB
*SFR* 000000CBH   DATA     BYTE      MD_MBH
*SFR* 000000CAH   DATA     BYTE      MD_MBL
*SFR* 000000C1H   DATA     BYTE      MD_MODE
*SFR* 00000098H.6 DATA     BIT       MOD0
*SFR* 00000098H.7 DATA     BIT       MOD1
*SFR* 000000F8H.7 DATA     BIT       MOE
*SFR* 000000F8H.6 DATA     BIT       OIS4
*SFR* 000000F8H   DATA     BIT       OISUH
*SFR* 000000F8H.1 DATA     BIT       OISUL
*SFR* 000000F8H.2 DATA     BIT       OISVH
*SFR* 000000F8H.3 DATA     BIT       OISVL
*SFR* 000000F8H.4 DATA     BIT       OISWH
*SFR* 000000F8H.5 DATA     BIT       OISWL
*SFR* 000000F1H   DATA     BYTE      OSC_CFG
*SFR* 000000D0H.2 DATA     BIT       OV
*SFR* 000000D0H   DATA     BIT       P
*SFR* 00000080H   DATA     BYTE      P0
*SFR* 000000FCH   DATA     BYTE      P0_OE
*SFR* 00000090H   DATA     BYTE      P1
*SFR* 000000FDH   DATA     BYTE      P1_OE
*SFR* 000000D1H   DATA     BYTE      P1IE
*SFR* 000000D2H   DATA     BYTE      P1IF
*SFR* 000000A0H   DATA     BYTE      P2
*SFR* 000000FEH   DATA     BYTE      P2_OE
*SFR* 000000D3H   DATA     BYTE      P2IE
*SFR* 000000D4H   DATA     BYTE      P2IF
*SFR* 000000B0H   DATA     BYTE      P3
*SFR* 000000FFH   DATA     BYTE      P3_OE
*SFR* 000000C0H.4 DATA     BIT       PADC0
*SFR* 000000C0H.5 DATA     BIT       PADC1
*SFR* 000000C0H.6 DATA     BIT       PCMP0
*SFR* 000000C0H.7 DATA     BIT       PCMP1
*SFR* 00000087H   DATA     BYTE      PCON
*SFR* 000000B8H.6 DATA     BIT       PFOC0
*SFR* 000000B8H.7 DATA     BIT       PFOC1
*SFR* 000000D8H.2 DATA     BIT       PI2C0
*SFR* 000000D8H.3 DATA     BIT       PI2C1
*SFR* 000000EAH   DATA     WORD      PI_EK
*SFR* 000000EBH   DATA     BYTE      PI_EKH
*SFR* 000000EAH   DATA     BYTE      PI_EKL
*SFR* 000000F2H   DATA     WORD      PI_KI
*SFR* 000000F3H   DATA     BYTE      PI_KIH
*SFR* 000000F2H   DATA     BYTE      PI_KIL
*SFR* 000000EEH   DATA     WORD      PI_KP
*SFR* 000000EFH   DATA     BYTE      PI_KPH
*SFR* 000000EEH   DATA     BYTE      PI_KPL
*SFR* 000000ECH   DATA     WORD      PI_UK
*SFR* 000000EDH   DATA     BYTE      PI_UKH
*SFR* 000000ECH   DATA     BYTE      PI_UKL
*SFR* 000000F4H   DATA     WORD      PI_UKMAX
LX51 LINKER/LOCATER V4.66.1.0                                                         07/21/2017  11:34:04  PAGE 5


*SFR* 000000F5H   DATA     BYTE      PI_UKMAXH
*SFR* 000000F4H   DATA     BYTE      PI_UKMAXL
*SFR* 000000F6H   DATA     WORD      PI_UKMIN
*SFR* 000000F7H   DATA     BYTE      PI_UKMINH
*SFR* 000000F6H   DATA     BYTE      PI_UKMINL
*SFR* 000000F9H   DATA     BYTE      PL_CR
*SFR* 000000B8H   DATA     BIT       PLVD0
*SFR* 000000B8H.1 DATA     BIT       PLVD1
*SFR* 000000D8H.6 DATA     BIT       PMCD0
*SFR* 000000D8H.7 DATA     BIT       PMCD1
*SFR* 000000C8H   DATA     BIT       PRTC0
*SFR* 000000C8H.1 DATA     BIT       PRTC1
*SFR* 00000085H   DATA     BYTE      PSCTL
*SFR* 000000D8H.4 DATA     BIT       PSPI0
*SFR* 000000D8H.5 DATA     BIT       PSPI1
*SFR* 000000D0H   DATA     BYTE      PSW
*SFR* 000000C0H   DATA     BIT       PTIM00
*SFR* 000000C0H.1 DATA     BIT       PTIM01
*SFR* 000000C0H.2 DATA     BIT       PTIM10
*SFR* 000000C0H.3 DATA     BIT       PTIM11
*SFR* 000000C8H.2 DATA     BIT       PTIM230
*SFR* 000000C8H.3 DATA     BIT       PTIM231
*SFR* 000000C8H.4 DATA     BIT       PTIM450
*SFR* 000000C8H.5 DATA     BIT       PTIM451
*SFR* 000000C8H.6 DATA     BIT       PTSD0
*SFR* 000000C8H.7 DATA     BIT       PTSD1
*SFR* 000000D8H   DATA     BIT       PUART0
*SFR* 000000D8H.1 DATA     BIT       PUART1
*SFR* 000000B8H.2 DATA     BIT       PX00
*SFR* 000000B8H.3 DATA     BIT       PX01
*SFR* 000000B8H.4 DATA     BIT       PX10
*SFR* 000000B8H.5 DATA     BIT       PX11
*SFR* 00000098H.2 DATA     BIT       RB8
*SFR* 00000098H.4 DATA     BIT       REN
*SFR* 00000098H   DATA     BIT       RI
*SFR* 000000D0H.3 DATA     BIT       RS0
*SFR* 000000D0H.4 DATA     BIT       RS1
*SFR* 000000C9H   DATA     BYTE      RSTSRC
*SFR* 000000A8H.6 DATA     BIT       RTCIE
*SFR* 00000098H.5 DATA     BIT       SM2
      0100014AH   CODE     ---       SoftwareInit
*SFR* 00000081H   DATA     BYTE      SP
*SFR* 000000A8H.3 DATA     BIT       SPIIE
*SFR* 000000E4H   DATA     WORD      SV_ANGLE
*SFR* 000000E5H   DATA     BYTE      SV_ANGLEH
*SFR* 000000E4H   DATA     BYTE      SV_ANGLEL
*SFR* 000000E1H   DATA     BYTE      SV_CR
*SFR* 000000E2H   DATA     WORD      SV_US
*SFR* 000000E3H   DATA     BYTE      SV_USH
*SFR* 000000E2H   DATA     BYTE      SV_USL
*SFR* 00000098H.3 DATA     BIT       TB8
*SFR* 00000088H   DATA     BYTE      TCON
*SFR* 00000098H.1 DATA     BIT       TI
*SFR* 000000B6H   DATA     WORD      TIM0_CCR1
*SFR* 000000B7H   DATA     BYTE      TIM0_CCR1H
*SFR* 000000B6H   DATA     BYTE      TIM0_CCR1L
*SFR* 000000BAH   DATA     WORD      TIM0_CCR2
*SFR* 000000BBH   DATA     BYTE      TIM0_CCR2H
*SFR* 000000BAH   DATA     BYTE      TIM0_CCR2L
*SFR* 000000BCH   DATA     WORD      TIM0_CCR3
*SFR* 000000BDH   DATA     BYTE      TIM0_CCR3H
*SFR* 000000BCH   DATA     BYTE      TIM0_CCR3L
*SFR* 000000BEH   DATA     WORD      TIM0_CCR4
*SFR* 000000BFH   DATA     BYTE      TIM0_CCR4H
*SFR* 000000BEH   DATA     BYTE      TIM0_CCR4L
LX51 LINKER/LOCATER V4.66.1.0                                                         07/21/2017  11:34:04  PAGE 6


*SFR* 000000B9H   DATA     BYTE      TIM0_IER
*SFR* 000000B1H   DATA     BYTE      TIM0_SR1
*SFR* 000000B4H   DATA     WORD      TIM2_ADTR
*SFR* 000000B5H   DATA     BYTE      TIM2_ADTRH
*SFR* 000000B4H   DATA     BYTE      TIM2_ADTRL
*SFR* 000000AEH   DATA     WORD      TIM2_ARR
*SFR* 000000AFH   DATA     BYTE      TIM2_ARRH
*SFR* 000000AEH   DATA     BYTE      TIM2_ARRL
*SFR* 000000B2H   DATA     WORD      TIM2_CMTR
*SFR* 000000B3H   DATA     BYTE      TIM2_CMTRH
*SFR* 000000B2H   DATA     BYTE      TIM2_CMTRL
*SFR* 000000AAH   DATA     WORD      TIM2_CNTR
*SFR* 000000ABH   DATA     BYTE      TIM2_CNTRH
*SFR* 000000AAH   DATA     BYTE      TIM2_CNTRL
*SFR* 000000A1H   DATA     BYTE      TIM2_CR0
*SFR* 000000A9H   DATA     BYTE      TIM2_CR1
*SFR* 000000ACH   DATA     WORD      TIM2_DR
*SFR* 000000ADH   DATA     BYTE      TIM2_DRH
*SFR* 000000ACH   DATA     BYTE      TIM2_DRL
*SFR* 000000A6H   DATA     WORD      TIM3_ARR
*SFR* 000000A7H   DATA     BYTE      TIM3_ARRH
*SFR* 000000A6H   DATA     BYTE      TIM3_ARRL
*SFR* 000000A2H   DATA     WORD      TIM3_CNTR
*SFR* 000000A3H   DATA     BYTE      TIM3_CNTRH
*SFR* 000000A2H   DATA     BYTE      TIM3_CNTRL
*SFR* 0000009CH   DATA     BYTE      TIM3_CR0
*SFR* 0000009DH   DATA     BYTE      TIM3_CR1
*SFR* 000000A4H   DATA     WORD      TIM3_DR
*SFR* 000000A5H   DATA     BYTE      TIM3_DRH
*SFR* 000000A4H   DATA     BYTE      TIM3_DRL
*SFR* 00000096H   DATA     WORD      TIM4_ARR
*SFR* 00000097H   DATA     BYTE      TIM4_ARRH
*SFR* 00000096H   DATA     BYTE      TIM4_ARRL
*SFR* 00000092H   DATA     WORD      TIM4_CNTR
*SFR* 00000093H   DATA     BYTE      TIM4_CNTRH
*SFR* 00000092H   DATA     BYTE      TIM4_CNTRL
*SFR* 0000009EH   DATA     BYTE      TIM4_CR0
*SFR* 0000009FH   DATA     BYTE      TIM4_CR1
*SFR* 00000094H   DATA     WORD      TIM4_DR
*SFR* 00000095H   DATA     BYTE      TIM4_DRH
*SFR* 00000094H   DATA     BYTE      TIM4_DRL
*SFR* 0000008EH   DATA     WORD      TIM5_ARR
*SFR* 0000008FH   DATA     BYTE      TIM5_ARRH
*SFR* 0000008EH   DATA     BYTE      TIM5_ARRL
*SFR* 0000008AH   DATA     WORD      TIM5_CNTR
*SFR* 0000008BH   DATA     BYTE      TIM5_CNTRH
*SFR* 0000008AH   DATA     BYTE      TIM5_CNTRL
*SFR* 00000089H   DATA     BYTE      TIM5_CR0
*SFR* 00000091H   DATA     BYTE      TIM5_CR1
*SFR* 0000008CH   DATA     WORD      TIM5_DR
*SFR* 0000008DH   DATA     BYTE      TIM5_DRH
*SFR* 0000008CH   DATA     BYTE      TIM5_DRL
*SFR* 000000A8H.1 DATA     BIT       TSDIE
*SFR* 00000088H.5 DATA     BIT       TSDIF
      01000121H   CODE     ---       UART_Init
      01000003H   CODE     ---       UART_ISR
      02000000H   XDATA    BYTE      UARTData
*SFR* 0000009AH   DATA     WORD      UT_BAUD
*SFR* 0000009BH   DATA     BYTE      UT_BAUDH
*SFR* 0000009AH   DATA     BYTE      UT_BAUDL
*SFR* 00000098H   DATA     BYTE      UT_CR
*SFR* 00000099H   DATA     BYTE      UT_DR



LX51 LINKER/LOCATER V4.66.1.0                                                         07/21/2017  11:34:04  PAGE 7


SYMBOL TABLE OF MODULE:  .\Output\FU68xx_UART_Demo (MAIN)

      VALUE       REP       CLASS    TYPE      SYMBOL NAME
      ====================================================
      ---         MODULE    ---      ---       MAIN
      0100014BH   PUBLIC    CODE     ---       HardwareInit
      0100014AH   PUBLIC    CODE     ---       SoftwareInit
      01000050H   PUBLIC    CODE     ---       main
      000000E2H   SFRSYM    DATA     BYTE      SV_USL
      000000ABH   SFRSYM    DATA     BYTE      TIM2_CNTRH
      000000B0H.4 SFRSYM    DATA     BIT       GP34
      000000A0H.5 SFRSYM    DATA     BIT       GP25
      00000090H.6 SFRSYM    DATA     BIT       GP16
      00000080H.7 SFRSYM    DATA     BIT       GP07
      00000088H.1 SFRSYM    DATA     BIT       IT01
      00000088H.3 SFRSYM    DATA     BIT       IT10
      000000F6H   SFRSYM    DATA     WORD      PI_UKMIN
      000000C2H   SFRSYM    DATA     WORD      MD_MA
      000000A3H   SFRSYM    DATA     BYTE      TIM3_CNTRH
      000000B0H.5 SFRSYM    DATA     BIT       GP35
      000000A0H.6 SFRSYM    DATA     BIT       GP26
      00000090H.7 SFRSYM    DATA     BIT       GP17
      00000080H   SFRSYM    DATA     BYTE      P0
      00000088H.4 SFRSYM    DATA     BIT       IT11
      000000CAH   SFRSYM    DATA     WORD      MD_MB
      00000093H   SFRSYM    DATA     BYTE      TIM4_CNTRH
      000000B0H.6 SFRSYM    DATA     BIT       GP36
      000000A0H.7 SFRSYM    DATA     BIT       GP27
      00000090H   SFRSYM    DATA     BYTE      P1
      000000D9H   SFRSYM    DATA     BYTE      EVT_FILT
      000000F4H   SFRSYM    DATA     WORD      PI_UKMAX
      0000008BH   SFRSYM    DATA     BYTE      TIM5_CNTRH
      000000B2H   SFRSYM    DATA     BYTE      TIM2_CMTRL
      000000B0H.7 SFRSYM    DATA     BIT       GP37
      000000A0H   SFRSYM    DATA     BYTE      P2
      000000AAH   SFRSYM    DATA     BYTE      TIM2_CNTRL
      000000B0H   SFRSYM    DATA     BYTE      P3
      000000A2H   SFRSYM    DATA     BYTE      TIM3_CNTRL
      000000D0H.6 SFRSYM    DATA     BIT       AC
      00000092H   SFRSYM    DATA     BYTE      TIM4_CNTRL
      0000008AH   SFRSYM    DATA     BYTE      TIM5_CNTRL
      000000B6H   SFRSYM    DATA     WORD      TIM0_CCR1
      000000A8H.7 SFRSYM    DATA     BIT       EA
      000000D5H   SFRSYM    DATA     BYTE      CMP_CR0
      000000BAH   SFRSYM    DATA     WORD      TIM0_CCR2
      000000D6H   SFRSYM    DATA     BYTE      CMP_CR1
      000000BCH   SFRSYM    DATA     WORD      TIM0_CCR3
      00000085H   SFRSYM    DATA     BYTE      PSCTL
      000000DAH   SFRSYM    DATA     BYTE      CMP_CR2
      000000BEH   SFRSYM    DATA     WORD      TIM0_CCR4
      000000B8H.2 SFRSYM    DATA     BIT       PX00
      000000EAH   SFRSYM    DATA     WORD      PI_EK
      000000F8H   SFRSYM    DATA     BIT       OISUH
      000000B8H.3 SFRSYM    DATA     BIT       PX01
      000000B8H.4 SFRSYM    DATA     BIT       PX10
      000000F8H.2 SFRSYM    DATA     BIT       OISVH
      000000B8H.5 SFRSYM    DATA     BIT       PX11
      000000F8H.4 SFRSYM    DATA     BIT       OISWH
      000000DCH   SFRSYM    DATA     WORD      LPF_K
      000000F2H   SFRSYM    DATA     WORD      PI_KI
      000000F8H.1 SFRSYM    DATA     BIT       OISUL
      000000A8H   SFRSYM    DATA     BYTE      IE
      000000F8H.3 SFRSYM    DATA     BIT       OISVL
      000000F8H.5 SFRSYM    DATA     BIT       OISWL
      000000D1H   SFRSYM    DATA     BYTE      P1IE
LX51 LINKER/LOCATER V4.66.1.0                                                         07/21/2017  11:34:04  PAGE 8


      00000098H.6 SFRSYM    DATA     BIT       MOD0
      000000D3H   SFRSYM    DATA     BYTE      P2IE
      000000D2H   SFRSYM    DATA     BYTE      P1IF
      000000F9H   SFRSYM    DATA     BYTE      PL_CR
      00000098H.7 SFRSYM    DATA     BIT       MOD1
      000000D4H   SFRSYM    DATA     BYTE      P2IF
      000000ACH   SFRSYM    DATA     WORD      TIM2_DR
      00000082H   SFRSYM    DATA     WORD      DP
      000000EEH   SFRSYM    DATA     WORD      PI_KP
      000000A4H   SFRSYM    DATA     WORD      TIM3_DR
      00000094H   SFRSYM    DATA     WORD      TIM4_DR
      0000008CH   SFRSYM    DATA     WORD      TIM5_DR
      000000F1H   SFRSYM    DATA     BYTE      OSC_CFG
      000000C1H   SFRSYM    DATA     BYTE      MD_MODE
      000000ECH   SFRSYM    DATA     WORD      PI_UK
      000000DEH   SFRSYM    DATA     WORD      LPF_X
      00000098H   SFRSYM    DATA     BIT       RI
      000000E6H   SFRSYM    DATA     WORD      LPF_Y
      000000C0H   SFRSYM    DATA     BIT       PTIM00
      000000D0H.7 SFRSYM    DATA     BIT       CY
      00000098H.1 SFRSYM    DATA     BIT       TI
      000000C0H.1 SFRSYM    DATA     BIT       PTIM01
      000000C0H.2 SFRSYM    DATA     BIT       PTIM10
      000000C0H.3 SFRSYM    DATA     BIT       PTIM11
      000000E1H   SFRSYM    DATA     BYTE      SV_CR
      00000098H   SFRSYM    DATA     BYTE      UT_CR
      00000099H   SFRSYM    DATA     BYTE      UT_DR
      000000F8H.6 SFRSYM    DATA     BIT       OIS4
      00000081H   SFRSYM    DATA     BYTE      SP
      000000D0H.2 SFRSYM    DATA     BIT       OV
      000000C4H   SFRSYM    DATA     BYTE      MD_DA0
      0000009AH   SFRSYM    DATA     WORD      UT_BAUD
      000000CCH   SFRSYM    DATA     BYTE      MD_DB0
      000000C5H   SFRSYM    DATA     BYTE      MD_DA1
      000000CDH   SFRSYM    DATA     BYTE      MD_DB1
      000000C6H   SFRSYM    DATA     BYTE      MD_DA2
      000000CEH   SFRSYM    DATA     BYTE      MD_DB2
      000000C7H   SFRSYM    DATA     BYTE      MD_DA3
      000000B4H   SFRSYM    DATA     WORD      TIM2_ADTR
      000000CFH   SFRSYM    DATA     BYTE      MD_DB3
      000000AFH   SFRSYM    DATA     BYTE      TIM2_ARRH
      000000A7H   SFRSYM    DATA     BYTE      TIM3_ARRH
      00000097H   SFRSYM    DATA     BYTE      TIM4_ARRH
      0000008FH   SFRSYM    DATA     BYTE      TIM5_ARRH
      000000AEH   SFRSYM    DATA     BYTE      TIM2_ARRL
      000000A6H   SFRSYM    DATA     BYTE      TIM3_ARRL
      00000087H   SFRSYM    DATA     BYTE      PCON
      000000E2H   SFRSYM    DATA     WORD      SV_US
      00000096H   SFRSYM    DATA     BYTE      TIM4_ARRL
      0000008EH   SFRSYM    DATA     BYTE      TIM5_ARRL
      000000B2H   SFRSYM    DATA     WORD      TIM2_CMTR
      00000088H   SFRSYM    DATA     BYTE      TCON
      000000AAH   SFRSYM    DATA     WORD      TIM2_CNTR
      000000A2H   SFRSYM    DATA     WORD      TIM3_CNTR
      00000092H   SFRSYM    DATA     WORD      TIM4_CNTR
      0000008AH   SFRSYM    DATA     WORD      TIM5_CNTR
      000000E5H   SFRSYM    DATA     BYTE      SV_ANGLEH
      00000086H   SFRSYM    DATA     BYTE      CFGKEY
      000000D8H   SFRSYM    DATA     BIT       PUART0
      000000E4H   SFRSYM    DATA     BYTE      SV_ANGLEL
      000000C6H   SFRSYM    DATA     WORD      MD_DAH
      000000D8H.1 SFRSYM    DATA     BIT       PUART1
      000000D8H.2 SFRSYM    DATA     BIT       PI2C0
      00000088H.2 SFRSYM    DATA     BIT       IF0
      000000CEH   SFRSYM    DATA     WORD      MD_DBH
LX51 LINKER/LOCATER V4.66.1.0                                                         07/21/2017  11:34:04  PAGE 9


      000000D8H.3 SFRSYM    DATA     BIT       PI2C1
      000000F0H   SFRSYM    DATA     BYTE      B
      000000C4H   SFRSYM    DATA     WORD      MD_DAL
      000000A1H   SFRSYM    DATA     BYTE      TIM2_CR0
      000000CCH   SFRSYM    DATA     WORD      MD_DBL
      0000009CH   SFRSYM    DATA     BYTE      TIM3_CR0
      000000A9H   SFRSYM    DATA     BYTE      TIM2_CR1
      0000009EH   SFRSYM    DATA     BYTE      TIM4_CR0
      0000009DH   SFRSYM    DATA     BYTE      TIM3_CR1
      00000089H   SFRSYM    DATA     BYTE      TIM5_CR0
      0000009FH   SFRSYM    DATA     BYTE      TIM4_CR1
      000000F8H   SFRSYM    DATA     BYTE      DRV_OUT
      00000091H   SFRSYM    DATA     BYTE      TIM5_CR1
      000000E0H   SFRSYM    DATA     BYTE      ACC
      000000F7H   SFRSYM    DATA     BYTE      PI_UKMINH
      000000C3H   SFRSYM    DATA     BYTE      MD_MAH
      000000A8H.4 SFRSYM    DATA     BIT       ES0
      000000DBH   SFRSYM    DATA     BYTE      LVSR
      000000CBH   SFRSYM    DATA     BYTE      MD_MBH
      000000C0H.4 SFRSYM    DATA     BIT       PADC0
      000000B8H   SFRSYM    DATA     BYTE      IP0
      000000F5H   SFRSYM    DATA     BYTE      PI_UKMAXH
      000000C0H.5 SFRSYM    DATA     BIT       PADC1
      000000C0H   SFRSYM    DATA     BYTE      IP1
      000000C8H   SFRSYM    DATA     BYTE      IP2
      000000F6H   SFRSYM    DATA     BYTE      PI_UKMINL
      000000C2H   SFRSYM    DATA     BYTE      MD_MAL
      00000098H.2 SFRSYM    DATA     BIT       RB8
      000000D8H   SFRSYM    DATA     BYTE      IP3
      000000CAH   SFRSYM    DATA     BYTE      MD_MBL
      000000A8H   SFRSYM    DATA     BIT       EX0
      000000F4H   SFRSYM    DATA     BYTE      PI_UKMAXL
      00000098H.3 SFRSYM    DATA     BIT       TB8
      000000B7H   SFRSYM    DATA     BYTE      TIM0_CCR1H
      000000A8H.2 SFRSYM    DATA     BIT       EX1
      000000BBH   SFRSYM    DATA     BYTE      TIM0_CCR2H
      000000D0H   SFRSYM    DATA     BIT       P
      000000BDH   SFRSYM    DATA     BYTE      TIM0_CCR3H
      000000BFH   SFRSYM    DATA     BYTE      TIM0_CCR4H
      000000C8H.2 SFRSYM    DATA     BIT       PTIM230
      000000EBH   SFRSYM    DATA     BYTE      PI_EKH
      00000098H.5 SFRSYM    DATA     BIT       SM2
      000000B6H   SFRSYM    DATA     BYTE      TIM0_CCR1L
      000000B1H   SFRSYM    DATA     BYTE      TIM0_SR1
      000000C8H.3 SFRSYM    DATA     BIT       PTIM231
      000000BAH   SFRSYM    DATA     BYTE      TIM0_CCR2L
      000000BCH   SFRSYM    DATA     BYTE      TIM0_CCR3L
      000000BEH   SFRSYM    DATA     BYTE      TIM0_CCR4L
      000000D8H.6 SFRSYM    DATA     BIT       PMCD0
      000000C8H.4 SFRSYM    DATA     BIT       PTIM450
      000000D0H.3 SFRSYM    DATA     BIT       RS0
      000000DDH   SFRSYM    DATA     BYTE      LPF_KH
      000000F3H   SFRSYM    DATA     BYTE      PI_KIH
      000000EAH   SFRSYM    DATA     BYTE      PI_EKL
      000000E8H   SFRSYM    DATA     BYTE      FOC_SET0
      000000D8H.7 SFRSYM    DATA     BIT       PMCD1
      000000C8H.5 SFRSYM    DATA     BIT       PTIM451
      000000D0H.4 SFRSYM    DATA     BIT       RS1
      000000E9H   SFRSYM    DATA     BYTE      FOC_SET1
      000000B8H.6 SFRSYM    DATA     BIT       PFOC0
      000000DCH   SFRSYM    DATA     BYTE      LPF_KL
      000000F2H   SFRSYM    DATA     BYTE      PI_KIL
      000000B8H.7 SFRSYM    DATA     BIT       PFOC1
      000000ADH   SFRSYM    DATA     BYTE      TIM2_DRH
      000000B9H   SFRSYM    DATA     BYTE      TIM0_IER
LX51 LINKER/LOCATER V4.66.1.0                                                         07/21/2017  11:34:04  PAGE 10


      00000083H   SFRSYM    DATA     BYTE      DPH
      000000EFH   SFRSYM    DATA     BYTE      PI_KPH
      000000A5H   SFRSYM    DATA     BYTE      TIM3_DRH
      00000095H   SFRSYM    DATA     BYTE      TIM4_DRH
      0000008DH   SFRSYM    DATA     BYTE      TIM5_DRH
      000000ACH   SFRSYM    DATA     BYTE      TIM2_DRL
      00000082H   SFRSYM    DATA     BYTE      DPL
      000000EEH   SFRSYM    DATA     BYTE      PI_KPL
      000000A4H   SFRSYM    DATA     BYTE      TIM3_DRL
      000000F8H.7 SFRSYM    DATA     BIT       MOE
      000000C0H.6 SFRSYM    DATA     BIT       PCMP0
      000000EDH   SFRSYM    DATA     BYTE      PI_UKH
      00000094H   SFRSYM    DATA     BYTE      TIM4_DRL
      000000C0H.7 SFRSYM    DATA     BIT       PCMP1
      000000DFH   SFRSYM    DATA     BYTE      LPF_XH
      0000008CH   SFRSYM    DATA     BYTE      TIM5_DRL
      000000AEH   SFRSYM    DATA     WORD      TIM2_ARR
      000000A8H.5 SFRSYM    DATA     BIT       MCDIE
      000000C9H   SFRSYM    DATA     BYTE      RSTSRC
      000000E7H   SFRSYM    DATA     BYTE      LPF_YH
      000000A6H   SFRSYM    DATA     WORD      TIM3_ARR
      00000088H.6 SFRSYM    DATA     BIT       MCDIF
      00000098H.4 SFRSYM    DATA     BIT       REN
      00000096H   SFRSYM    DATA     WORD      TIM4_ARR
      000000ECH   SFRSYM    DATA     BYTE      PI_UKL
      000000D7H   SFRSYM    DATA     BYTE      CMP_SR
      0000008EH   SFRSYM    DATA     WORD      TIM5_ARR
      000000DEH   SFRSYM    DATA     BYTE      LPF_XL
      000000B8H   SFRSYM    DATA     BIT       PLVD0
      000000E6H   SFRSYM    DATA     BYTE      LPF_YL
      000000B8H.1 SFRSYM    DATA     BIT       PLVD1
      000000C8H   SFRSYM    DATA     BIT       PRTC0
      000000C8H.1 SFRSYM    DATA     BIT       PRTC1
      000000E8H.7 SFRSYM    DATA     BIT       FOCEN
      000000C8H.6 SFRSYM    DATA     BIT       PTSD0
      000000D8H.4 SFRSYM    DATA     BIT       PSPI0
      000000C8H.7 SFRSYM    DATA     BIT       PTSD1
      000000D8H.5 SFRSYM    DATA     BIT       PSPI1
      0000009BH   SFRSYM    DATA     BYTE      UT_BAUDH
      000000E4H   SFRSYM    DATA     WORD      SV_ANGLE
      000000B5H   SFRSYM    DATA     BYTE      TIM2_ADTRH
      0000009AH   SFRSYM    DATA     BYTE      UT_BAUDL
      000000FCH   SFRSYM    DATA     BYTE      P0_OE
      000000FDH   SFRSYM    DATA     BYTE      P1_OE
      000000D0H.5 SFRSYM    DATA     BIT       F0
      000000B4H   SFRSYM    DATA     BYTE      TIM2_ADTRL
      000000FEH   SFRSYM    DATA     BYTE      P2_OE
      000000D0H.1 SFRSYM    DATA     BIT       F1
      00000080H   SFRSYM    DATA     BIT       GP00
      000000FFH   SFRSYM    DATA     BYTE      P3_OE
      00000090H   SFRSYM    DATA     BIT       GP10
      00000080H.1 SFRSYM    DATA     BIT       GP01
      000000A8H.6 SFRSYM    DATA     BIT       RTCIE
      000000A0H   SFRSYM    DATA     BIT       GP20
      00000090H.1 SFRSYM    DATA     BIT       GP11
      00000080H.2 SFRSYM    DATA     BIT       GP02
      000000E3H   SFRSYM    DATA     BYTE      SV_USH
      000000B0H   SFRSYM    DATA     BIT       GP30
      000000A0H.1 SFRSYM    DATA     BIT       GP21
      00000090H.2 SFRSYM    DATA     BIT       GP12
      00000080H.3 SFRSYM    DATA     BIT       GP03
      000000A8H.1 SFRSYM    DATA     BIT       TSDIE
      000000D0H   SFRSYM    DATA     BYTE      PSW
      000000B0H.1 SFRSYM    DATA     BIT       GP31
      000000A0H.2 SFRSYM    DATA     BIT       GP22
LX51 LINKER/LOCATER V4.66.1.0                                                         07/21/2017  11:34:04  PAGE 11


      00000090H.3 SFRSYM    DATA     BIT       GP13
      00000080H.4 SFRSYM    DATA     BIT       GP04
      000000A8H.3 SFRSYM    DATA     BIT       SPIIE
      00000088H.5 SFRSYM    DATA     BIT       TSDIF
      000000B0H.2 SFRSYM    DATA     BIT       GP32
      000000A0H.3 SFRSYM    DATA     BIT       GP23
      00000090H.4 SFRSYM    DATA     BIT       GP14
      00000080H.5 SFRSYM    DATA     BIT       GP05
      00000084H   SFRSYM    DATA     BYTE      FLKEY
      000000B3H   SFRSYM    DATA     BYTE      TIM2_CMTRH
      000000B0H.3 SFRSYM    DATA     BIT       GP33
      000000A0H.4 SFRSYM    DATA     BIT       GP24
      00000090H.5 SFRSYM    DATA     BIT       GP15
      00000080H.6 SFRSYM    DATA     BIT       GP06
      00000088H   SFRSYM    DATA     BIT       IT00

      01000050H   BLOCK     CODE     ---       LVL=0
      01000050H   LINE      CODE     ---       #37
      01000050H   LINE      CODE     ---       #38
      01000050H   LINE      CODE     ---       #40
      01000053H   LINE      CODE     ---       #42
      01000056H   LINE      CODE     ---       #43
      01000059H   LINE      CODE     ---       #45
      01000059H   LINE      CODE     ---       #46
      01000059H   LINE      CODE     ---       #48
      ---         BLOCKEND  ---      ---       LVL=0

      0100014AH   BLOCK     CODE     ---       LVL=0
      0100014AH   LINE      CODE     ---       #58
      0100014AH   LINE      CODE     ---       #59
      0100014AH   LINE      CODE     ---       #61
      ---         BLOCKEND  ---      ---       LVL=0

      0100014BH   BLOCK     CODE     ---       LVL=0
      0100014BH   LINE      CODE     ---       #69
      0100014BH   LINE      CODE     ---       #70
      0100014BH   LINE      CODE     ---       #72
      ---         BLOCKEND  ---      ---       LVL=0

      ---         MODULE    ---      ---       INTERRUPT
      02000000H   PUBLIC    XDATA    BYTE      UARTData
      01000003H   PUBLIC    CODE     ---       UART_ISR
      000000E2H   SFRSYM    DATA     BYTE      SV_USL
      000000ABH   SFRSYM    DATA     BYTE      TIM2_CNTRH
      000000B0H.4 SFRSYM    DATA     BIT       GP34
      000000A0H.5 SFRSYM    DATA     BIT       GP25
      00000090H.6 SFRSYM    DATA     BIT       GP16
      00000080H.7 SFRSYM    DATA     BIT       GP07
      00000088H.1 SFRSYM    DATA     BIT       IT01
      00000088H.3 SFRSYM    DATA     BIT       IT10
      000000F6H   SFRSYM    DATA     WORD      PI_UKMIN
      000000C2H   SFRSYM    DATA     WORD      MD_MA
      000000A3H   SFRSYM    DATA     BYTE      TIM3_CNTRH
      000000B0H.5 SFRSYM    DATA     BIT       GP35
      000000A0H.6 SFRSYM    DATA     BIT       GP26
      00000090H.7 SFRSYM    DATA     BIT       GP17
      00000080H   SFRSYM    DATA     BYTE      P0
      00000088H.4 SFRSYM    DATA     BIT       IT11
      000000CAH   SFRSYM    DATA     WORD      MD_MB
      00000093H   SFRSYM    DATA     BYTE      TIM4_CNTRH
      000000B0H.6 SFRSYM    DATA     BIT       GP36
      000000A0H.7 SFRSYM    DATA     BIT       GP27
      00000090H   SFRSYM    DATA     BYTE      P1
      000000D9H   SFRSYM    DATA     BYTE      EVT_FILT
      000000F4H   SFRSYM    DATA     WORD      PI_UKMAX
LX51 LINKER/LOCATER V4.66.1.0                                                         07/21/2017  11:34:04  PAGE 12


      0000008BH   SFRSYM    DATA     BYTE      TIM5_CNTRH
      000000B2H   SFRSYM    DATA     BYTE      TIM2_CMTRL
      000000B0H.7 SFRSYM    DATA     BIT       GP37
      000000A0H   SFRSYM    DATA     BYTE      P2
      000000AAH   SFRSYM    DATA     BYTE      TIM2_CNTRL
      000000B0H   SFRSYM    DATA     BYTE      P3
      000000A2H   SFRSYM    DATA     BYTE      TIM3_CNTRL
      000000D0H.6 SFRSYM    DATA     BIT       AC
      00000092H   SFRSYM    DATA     BYTE      TIM4_CNTRL
      0000008AH   SFRSYM    DATA     BYTE      TIM5_CNTRL
      000000B6H   SFRSYM    DATA     WORD      TIM0_CCR1
      000000A8H.7 SFRSYM    DATA     BIT       EA
      000000D5H   SFRSYM    DATA     BYTE      CMP_CR0
      000000BAH   SFRSYM    DATA     WORD      TIM0_CCR2
      000000D6H   SFRSYM    DATA     BYTE      CMP_CR1
      000000BCH   SFRSYM    DATA     WORD      TIM0_CCR3
      00000085H   SFRSYM    DATA     BYTE      PSCTL
      000000DAH   SFRSYM    DATA     BYTE      CMP_CR2
      000000BEH   SFRSYM    DATA     WORD      TIM0_CCR4
      000000B8H.2 SFRSYM    DATA     BIT       PX00
      000000EAH   SFRSYM    DATA     WORD      PI_EK
      000000F8H   SFRSYM    DATA     BIT       OISUH
      000000B8H.3 SFRSYM    DATA     BIT       PX01
      000000B8H.4 SFRSYM    DATA     BIT       PX10
      000000F8H.2 SFRSYM    DATA     BIT       OISVH
      000000B8H.5 SFRSYM    DATA     BIT       PX11
      000000F8H.4 SFRSYM    DATA     BIT       OISWH
      000000DCH   SFRSYM    DATA     WORD      LPF_K
      000000F2H   SFRSYM    DATA     WORD      PI_KI
      000000F8H.1 SFRSYM    DATA     BIT       OISUL
      000000A8H   SFRSYM    DATA     BYTE      IE
      000000F8H.3 SFRSYM    DATA     BIT       OISVL
      000000F8H.5 SFRSYM    DATA     BIT       OISWL
      000000D1H   SFRSYM    DATA     BYTE      P1IE
      00000098H.6 SFRSYM    DATA     BIT       MOD0
      000000D3H   SFRSYM    DATA     BYTE      P2IE
      000000D2H   SFRSYM    DATA     BYTE      P1IF
      000000F9H   SFRSYM    DATA     BYTE      PL_CR
      00000098H.7 SFRSYM    DATA     BIT       MOD1
      000000D4H   SFRSYM    DATA     BYTE      P2IF
      000000ACH   SFRSYM    DATA     WORD      TIM2_DR
      00000082H   SFRSYM    DATA     WORD      DP
      000000EEH   SFRSYM    DATA     WORD      PI_KP
      000000A4H   SFRSYM    DATA     WORD      TIM3_DR
      00000094H   SFRSYM    DATA     WORD      TIM4_DR
      0000008CH   SFRSYM    DATA     WORD      TIM5_DR
      000000F1H   SFRSYM    DATA     BYTE      OSC_CFG
      000000C1H   SFRSYM    DATA     BYTE      MD_MODE
      000000ECH   SFRSYM    DATA     WORD      PI_UK
      000000DEH   SFRSYM    DATA     WORD      LPF_X
      00000098H   SFRSYM    DATA     BIT       RI
      000000E6H   SFRSYM    DATA     WORD      LPF_Y
      000000C0H   SFRSYM    DATA     BIT       PTIM00
      000000D0H.7 SFRSYM    DATA     BIT       CY
      00000098H.1 SFRSYM    DATA     BIT       TI
      000000C0H.1 SFRSYM    DATA     BIT       PTIM01
      000000C0H.2 SFRSYM    DATA     BIT       PTIM10
      000000C0H.3 SFRSYM    DATA     BIT       PTIM11
      000000E1H   SFRSYM    DATA     BYTE      SV_CR
      00000098H   SFRSYM    DATA     BYTE      UT_CR
      00000099H   SFRSYM    DATA     BYTE      UT_DR
      000000F8H.6 SFRSYM    DATA     BIT       OIS4
      00000081H   SFRSYM    DATA     BYTE      SP
      000000D0H.2 SFRSYM    DATA     BIT       OV
      000000C4H   SFRSYM    DATA     BYTE      MD_DA0
LX51 LINKER/LOCATER V4.66.1.0                                                         07/21/2017  11:34:04  PAGE 13


      0000009AH   SFRSYM    DATA     WORD      UT_BAUD
      000000CCH   SFRSYM    DATA     BYTE      MD_DB0
      000000C5H   SFRSYM    DATA     BYTE      MD_DA1
      000000CDH   SFRSYM    DATA     BYTE      MD_DB1
      000000C6H   SFRSYM    DATA     BYTE      MD_DA2
      000000CEH   SFRSYM    DATA     BYTE      MD_DB2
      000000C7H   SFRSYM    DATA     BYTE      MD_DA3
      000000B4H   SFRSYM    DATA     WORD      TIM2_ADTR
      000000CFH   SFRSYM    DATA     BYTE      MD_DB3
      000000AFH   SFRSYM    DATA     BYTE      TIM2_ARRH
      000000A7H   SFRSYM    DATA     BYTE      TIM3_ARRH
      00000097H   SFRSYM    DATA     BYTE      TIM4_ARRH
      0000008FH   SFRSYM    DATA     BYTE      TIM5_ARRH
      000000AEH   SFRSYM    DATA     BYTE      TIM2_ARRL
      000000A6H   SFRSYM    DATA     BYTE      TIM3_ARRL
      00000087H   SFRSYM    DATA     BYTE      PCON
      000000E2H   SFRSYM    DATA     WORD      SV_US
      00000096H   SFRSYM    DATA     BYTE      TIM4_ARRL
      0000008EH   SFRSYM    DATA     BYTE      TIM5_ARRL
      000000B2H   SFRSYM    DATA     WORD      TIM2_CMTR
      00000088H   SFRSYM    DATA     BYTE      TCON
      000000AAH   SFRSYM    DATA     WORD      TIM2_CNTR
      000000A2H   SFRSYM    DATA     WORD      TIM3_CNTR
      00000092H   SFRSYM    DATA     WORD      TIM4_CNTR
      0000008AH   SFRSYM    DATA     WORD      TIM5_CNTR
      000000E5H   SFRSYM    DATA     BYTE      SV_ANGLEH
      00000086H   SFRSYM    DATA     BYTE      CFGKEY
      000000D8H   SFRSYM    DATA     BIT       PUART0
      000000E4H   SFRSYM    DATA     BYTE      SV_ANGLEL
      000000C6H   SFRSYM    DATA     WORD      MD_DAH
      000000D8H.1 SFRSYM    DATA     BIT       PUART1
      000000D8H.2 SFRSYM    DATA     BIT       PI2C0
      00000088H.2 SFRSYM    DATA     BIT       IF0
      000000CEH   SFRSYM    DATA     WORD      MD_DBH
      000000D8H.3 SFRSYM    DATA     BIT       PI2C1
      000000F0H   SFRSYM    DATA     BYTE      B
      000000C4H   SFRSYM    DATA     WORD      MD_DAL
      000000A1H   SFRSYM    DATA     BYTE      TIM2_CR0
      000000CCH   SFRSYM    DATA     WORD      MD_DBL
      0000009CH   SFRSYM    DATA     BYTE      TIM3_CR0
      000000A9H   SFRSYM    DATA     BYTE      TIM2_CR1
      0000009EH   SFRSYM    DATA     BYTE      TIM4_CR0
      0000009DH   SFRSYM    DATA     BYTE      TIM3_CR1
      00000089H   SFRSYM    DATA     BYTE      TIM5_CR0
      0000009FH   SFRSYM    DATA     BYTE      TIM4_CR1
      000000F8H   SFRSYM    DATA     BYTE      DRV_OUT
      00000091H   SFRSYM    DATA     BYTE      TIM5_CR1
      000000E0H   SFRSYM    DATA     BYTE      ACC
      000000F7H   SFRSYM    DATA     BYTE      PI_UKMINH
      000000C3H   SFRSYM    DATA     BYTE      MD_MAH
      000000A8H.4 SFRSYM    DATA     BIT       ES0
      000000DBH   SFRSYM    DATA     BYTE      LVSR
      000000CBH   SFRSYM    DATA     BYTE      MD_MBH
      000000C0H.4 SFRSYM    DATA     BIT       PADC0
      000000B8H   SFRSYM    DATA     BYTE      IP0
      000000F5H   SFRSYM    DATA     BYTE      PI_UKMAXH
      000000C0H.5 SFRSYM    DATA     BIT       PADC1
      000000C0H   SFRSYM    DATA     BYTE      IP1
      000000C8H   SFRSYM    DATA     BYTE      IP2
      000000F6H   SFRSYM    DATA     BYTE      PI_UKMINL
      000000C2H   SFRSYM    DATA     BYTE      MD_MAL
      00000098H.2 SFRSYM    DATA     BIT       RB8
      000000D8H   SFRSYM    DATA     BYTE      IP3
      000000CAH   SFRSYM    DATA     BYTE      MD_MBL
      000000A8H   SFRSYM    DATA     BIT       EX0
LX51 LINKER/LOCATER V4.66.1.0                                                         07/21/2017  11:34:04  PAGE 14


      000000F4H   SFRSYM    DATA     BYTE      PI_UKMAXL
      00000098H.3 SFRSYM    DATA     BIT       TB8
      000000B7H   SFRSYM    DATA     BYTE      TIM0_CCR1H
      000000A8H.2 SFRSYM    DATA     BIT       EX1
      000000BBH   SFRSYM    DATA     BYTE      TIM0_CCR2H
      000000D0H   SFRSYM    DATA     BIT       P
      000000BDH   SFRSYM    DATA     BYTE      TIM0_CCR3H
      000000BFH   SFRSYM    DATA     BYTE      TIM0_CCR4H
      000000C8H.2 SFRSYM    DATA     BIT       PTIM230
      000000EBH   SFRSYM    DATA     BYTE      PI_EKH
      00000098H.5 SFRSYM    DATA     BIT       SM2
      000000B6H   SFRSYM    DATA     BYTE      TIM0_CCR1L
      000000B1H   SFRSYM    DATA     BYTE      TIM0_SR1
      000000C8H.3 SFRSYM    DATA     BIT       PTIM231
      000000BAH   SFRSYM    DATA     BYTE      TIM0_CCR2L
      000000BCH   SFRSYM    DATA     BYTE      TIM0_CCR3L
      000000BEH   SFRSYM    DATA     BYTE      TIM0_CCR4L
      000000D8H.6 SFRSYM    DATA     BIT       PMCD0
      000000C8H.4 SFRSYM    DATA     BIT       PTIM450
      000000D0H.3 SFRSYM    DATA     BIT       RS0
      000000DDH   SFRSYM    DATA     BYTE      LPF_KH
      000000F3H   SFRSYM    DATA     BYTE      PI_KIH
      000000EAH   SFRSYM    DATA     BYTE      PI_EKL
      000000E8H   SFRSYM    DATA     BYTE      FOC_SET0
      000000D8H.7 SFRSYM    DATA     BIT       PMCD1
      000000C8H.5 SFRSYM    DATA     BIT       PTIM451
      000000D0H.4 SFRSYM    DATA     BIT       RS1
      000000E9H   SFRSYM    DATA     BYTE      FOC_SET1
      000000B8H.6 SFRSYM    DATA     BIT       PFOC0
      000000DCH   SFRSYM    DATA     BYTE      LPF_KL
      000000F2H   SFRSYM    DATA     BYTE      PI_KIL
      000000B8H.7 SFRSYM    DATA     BIT       PFOC1
      000000ADH   SFRSYM    DATA     BYTE      TIM2_DRH
      000000B9H   SFRSYM    DATA     BYTE      TIM0_IER
      00000083H   SFRSYM    DATA     BYTE      DPH
      000000EFH   SFRSYM    DATA     BYTE      PI_KPH
      000000A5H   SFRSYM    DATA     BYTE      TIM3_DRH
      00000095H   SFRSYM    DATA     BYTE      TIM4_DRH
      0000008DH   SFRSYM    DATA     BYTE      TIM5_DRH
      000000ACH   SFRSYM    DATA     BYTE      TIM2_DRL
      00000082H   SFRSYM    DATA     BYTE      DPL
      000000EEH   SFRSYM    DATA     BYTE      PI_KPL
      000000A4H   SFRSYM    DATA     BYTE      TIM3_DRL
      000000F8H.7 SFRSYM    DATA     BIT       MOE
      000000C0H.6 SFRSYM    DATA     BIT       PCMP0
      000000EDH   SFRSYM    DATA     BYTE      PI_UKH
      00000094H   SFRSYM    DATA     BYTE      TIM4_DRL
      000000C0H.7 SFRSYM    DATA     BIT       PCMP1
      000000DFH   SFRSYM    DATA     BYTE      LPF_XH
      0000008CH   SFRSYM    DATA     BYTE      TIM5_DRL
      000000AEH   SFRSYM    DATA     WORD      TIM2_ARR
      000000A8H.5 SFRSYM    DATA     BIT       MCDIE
      000000C9H   SFRSYM    DATA     BYTE      RSTSRC
      000000E7H   SFRSYM    DATA     BYTE      LPF_YH
      000000A6H   SFRSYM    DATA     WORD      TIM3_ARR
      00000088H.6 SFRSYM    DATA     BIT       MCDIF
      00000098H.4 SFRSYM    DATA     BIT       REN
      00000096H   SFRSYM    DATA     WORD      TIM4_ARR
      000000ECH   SFRSYM    DATA     BYTE      PI_UKL
      000000D7H   SFRSYM    DATA     BYTE      CMP_SR
      0000008EH   SFRSYM    DATA     WORD      TIM5_ARR
      000000DEH   SFRSYM    DATA     BYTE      LPF_XL
      000000B8H   SFRSYM    DATA     BIT       PLVD0
      000000E6H   SFRSYM    DATA     BYTE      LPF_YL
      000000B8H.1 SFRSYM    DATA     BIT       PLVD1
LX51 LINKER/LOCATER V4.66.1.0                                                         07/21/2017  11:34:04  PAGE 15


      000000C8H   SFRSYM    DATA     BIT       PRTC0
      000000C8H.1 SFRSYM    DATA     BIT       PRTC1
      000000E8H.7 SFRSYM    DATA     BIT       FOCEN
      000000C8H.6 SFRSYM    DATA     BIT       PTSD0
      000000D8H.4 SFRSYM    DATA     BIT       PSPI0
      000000C8H.7 SFRSYM    DATA     BIT       PTSD1
      000000D8H.5 SFRSYM    DATA     BIT       PSPI1
      0000009BH   SFRSYM    DATA     BYTE      UT_BAUDH
      000000E4H   SFRSYM    DATA     WORD      SV_ANGLE
      000000B5H   SFRSYM    DATA     BYTE      TIM2_ADTRH
      0000009AH   SFRSYM    DATA     BYTE      UT_BAUDL
      000000FCH   SFRSYM    DATA     BYTE      P0_OE
      000000FDH   SFRSYM    DATA     BYTE      P1_OE
      000000D0H.5 SFRSYM    DATA     BIT       F0
      000000B4H   SFRSYM    DATA     BYTE      TIM2_ADTRL
      000000FEH   SFRSYM    DATA     BYTE      P2_OE
      000000D0H.1 SFRSYM    DATA     BIT       F1
      00000080H   SFRSYM    DATA     BIT       GP00
      000000FFH   SFRSYM    DATA     BYTE      P3_OE
      00000090H   SFRSYM    DATA     BIT       GP10
      00000080H.1 SFRSYM    DATA     BIT       GP01
      000000A8H.6 SFRSYM    DATA     BIT       RTCIE
      000000A0H   SFRSYM    DATA     BIT       GP20
      00000090H.1 SFRSYM    DATA     BIT       GP11
      00000080H.2 SFRSYM    DATA     BIT       GP02
      000000E3H   SFRSYM    DATA     BYTE      SV_USH
      000000B0H   SFRSYM    DATA     BIT       GP30
      000000A0H.1 SFRSYM    DATA     BIT       GP21
      00000090H.2 SFRSYM    DATA     BIT       GP12
      00000080H.3 SFRSYM    DATA     BIT       GP03
      000000A8H.1 SFRSYM    DATA     BIT       TSDIE
      000000D0H   SFRSYM    DATA     BYTE      PSW
      000000B0H.1 SFRSYM    DATA     BIT       GP31
      000000A0H.2 SFRSYM    DATA     BIT       GP22
      00000090H.3 SFRSYM    DATA     BIT       GP13
      00000080H.4 SFRSYM    DATA     BIT       GP04
      000000A8H.3 SFRSYM    DATA     BIT       SPIIE
      00000088H.5 SFRSYM    DATA     BIT       TSDIF
      000000B0H.2 SFRSYM    DATA     BIT       GP32
      000000A0H.3 SFRSYM    DATA     BIT       GP23
      00000090H.4 SFRSYM    DATA     BIT       GP14
      00000080H.5 SFRSYM    DATA     BIT       GP05
      00000084H   SFRSYM    DATA     BYTE      FLKEY
      000000B3H   SFRSYM    DATA     BYTE      TIM2_CMTRH
      000000B0H.3 SFRSYM    DATA     BIT       GP33
      000000A0H.4 SFRSYM    DATA     BIT       GP24
      00000090H.5 SFRSYM    DATA     BIT       GP15
      00000080H.6 SFRSYM    DATA     BIT       GP06
      00000088H   SFRSYM    DATA     BIT       IT00

      01000003H   BLOCK     CODE     ---       LVL=0
      01000003H   LINE      CODE     ---       #24
      01000020H   LINE      CODE     ---       #27
      01000023H   LINE      CODE     ---       #28
      01000023H   LINE      CODE     ---       #29
      01000025H   LINE      CODE     ---       #31
      0100002BH   LINE      CODE     ---       #33
      01000030H   LINE      CODE     ---       #35
      01000030H   LINE      CODE     ---       #38
      01000033H   LINE      CODE     ---       #39
      01000033H   LINE      CODE     ---       #40
      01000035H   LINE      CODE     ---       #41
      01000035H   LINE      CODE     ---       #43
      ---         BLOCKEND  ---      ---       LVL=0

LX51 LINKER/LOCATER V4.66.1.0                                                         07/21/2017  11:34:04  PAGE 16


      ---         MODULE    ---      ---       UARTINIT
      0100005BH   PUBLIC    CODE     ---       _UART_SendData
      01000121H   PUBLIC    CODE     ---       UART_Init
      000000E2H   SFRSYM    DATA     BYTE      SV_USL
      000000ABH   SFRSYM    DATA     BYTE      TIM2_CNTRH
      000000B0H.4 SFRSYM    DATA     BIT       GP34
      000000A0H.5 SFRSYM    DATA     BIT       GP25
      00000090H.6 SFRSYM    DATA     BIT       GP16
      00000080H.7 SFRSYM    DATA     BIT       GP07
      00000088H.1 SFRSYM    DATA     BIT       IT01
      00000088H.3 SFRSYM    DATA     BIT       IT10
      000000F6H   SFRSYM    DATA     WORD      PI_UKMIN
      000000C2H   SFRSYM    DATA     WORD      MD_MA
      000000A3H   SFRSYM    DATA     BYTE      TIM3_CNTRH
      000000B0H.5 SFRSYM    DATA     BIT       GP35
      000000A0H.6 SFRSYM    DATA     BIT       GP26
      00000090H.7 SFRSYM    DATA     BIT       GP17
      00000080H   SFRSYM    DATA     BYTE      P0
      00000088H.4 SFRSYM    DATA     BIT       IT11
      000000CAH   SFRSYM    DATA     WORD      MD_MB
      00000093H   SFRSYM    DATA     BYTE      TIM4_CNTRH
      000000B0H.6 SFRSYM    DATA     BIT       GP36
      000000A0H.7 SFRSYM    DATA     BIT       GP27
      00000090H   SFRSYM    DATA     BYTE      P1
      000000D9H   SFRSYM    DATA     BYTE      EVT_FILT
      000000F4H   SFRSYM    DATA     WORD      PI_UKMAX
      0000008BH   SFRSYM    DATA     BYTE      TIM5_CNTRH
      000000B2H   SFRSYM    DATA     BYTE      TIM2_CMTRL
      000000B0H.7 SFRSYM    DATA     BIT       GP37
      000000A0H   SFRSYM    DATA     BYTE      P2
      000000AAH   SFRSYM    DATA     BYTE      TIM2_CNTRL
      000000B0H   SFRSYM    DATA     BYTE      P3
      000000A2H   SFRSYM    DATA     BYTE      TIM3_CNTRL
      000000D0H.6 SFRSYM    DATA     BIT       AC
      00000092H   SFRSYM    DATA     BYTE      TIM4_CNTRL
      0000008AH   SFRSYM    DATA     BYTE      TIM5_CNTRL
      000000B6H   SFRSYM    DATA     WORD      TIM0_CCR1
      000000A8H.7 SFRSYM    DATA     BIT       EA
      000000D5H   SFRSYM    DATA     BYTE      CMP_CR0
      000000BAH   SFRSYM    DATA     WORD      TIM0_CCR2
      000000D6H   SFRSYM    DATA     BYTE      CMP_CR1
      000000BCH   SFRSYM    DATA     WORD      TIM0_CCR3
      00000085H   SFRSYM    DATA     BYTE      PSCTL
      000000DAH   SFRSYM    DATA     BYTE      CMP_CR2
      000000BEH   SFRSYM    DATA     WORD      TIM0_CCR4
      000000B8H.2 SFRSYM    DATA     BIT       PX00
      000000EAH   SFRSYM    DATA     WORD      PI_EK
      000000F8H   SFRSYM    DATA     BIT       OISUH
      000000B8H.3 SFRSYM    DATA     BIT       PX01
      000000B8H.4 SFRSYM    DATA     BIT       PX10
      000000F8H.2 SFRSYM    DATA     BIT       OISVH
      000000B8H.5 SFRSYM    DATA     BIT       PX11
      000000F8H.4 SFRSYM    DATA     BIT       OISWH
      000000DCH   SFRSYM    DATA     WORD      LPF_K
      000000F2H   SFRSYM    DATA     WORD      PI_KI
      000000F8H.1 SFRSYM    DATA     BIT       OISUL
      000000A8H   SFRSYM    DATA     BYTE      IE
      000000F8H.3 SFRSYM    DATA     BIT       OISVL
      000000F8H.5 SFRSYM    DATA     BIT       OISWL
      000000D1H   SFRSYM    DATA     BYTE      P1IE
      00000098H.6 SFRSYM    DATA     BIT       MOD0
      000000D3H   SFRSYM    DATA     BYTE      P2IE
      000000D2H   SFRSYM    DATA     BYTE      P1IF
      000000F9H   SFRSYM    DATA     BYTE      PL_CR
      00000098H.7 SFRSYM    DATA     BIT       MOD1
LX51 LINKER/LOCATER V4.66.1.0                                                         07/21/2017  11:34:04  PAGE 17


      000000D4H   SFRSYM    DATA     BYTE      P2IF
      000000ACH   SFRSYM    DATA     WORD      TIM2_DR
      00000082H   SFRSYM    DATA     WORD      DP
      000000EEH   SFRSYM    DATA     WORD      PI_KP
      000000A4H   SFRSYM    DATA     WORD      TIM3_DR
      00000094H   SFRSYM    DATA     WORD      TIM4_DR
      0000008CH   SFRSYM    DATA     WORD      TIM5_DR
      000000F1H   SFRSYM    DATA     BYTE      OSC_CFG
      000000C1H   SFRSYM    DATA     BYTE      MD_MODE
      000000ECH   SFRSYM    DATA     WORD      PI_UK
      000000DEH   SFRSYM    DATA     WORD      LPF_X
      00000098H   SFRSYM    DATA     BIT       RI
      000000E6H   SFRSYM    DATA     WORD      LPF_Y
      000000C0H   SFRSYM    DATA     BIT       PTIM00
      000000D0H.7 SFRSYM    DATA     BIT       CY
      00000098H.1 SFRSYM    DATA     BIT       TI
      000000C0H.1 SFRSYM    DATA     BIT       PTIM01
      000000C0H.2 SFRSYM    DATA     BIT       PTIM10
      000000C0H.3 SFRSYM    DATA     BIT       PTIM11
      000000E1H   SFRSYM    DATA     BYTE      SV_CR
      00000098H   SFRSYM    DATA     BYTE      UT_CR
      00000099H   SFRSYM    DATA     BYTE      UT_DR
      000000F8H.6 SFRSYM    DATA     BIT       OIS4
      00000081H   SFRSYM    DATA     BYTE      SP
      000000D0H.2 SFRSYM    DATA     BIT       OV
      000000C4H   SFRSYM    DATA     BYTE      MD_DA0
      0000009AH   SFRSYM    DATA     WORD      UT_BAUD
      000000CCH   SFRSYM    DATA     BYTE      MD_DB0
      000000C5H   SFRSYM    DATA     BYTE      MD_DA1
      000000CDH   SFRSYM    DATA     BYTE      MD_DB1
      000000C6H   SFRSYM    DATA     BYTE      MD_DA2
      000000CEH   SFRSYM    DATA     BYTE      MD_DB2
      000000C7H   SFRSYM    DATA     BYTE      MD_DA3
      000000B4H   SFRSYM    DATA     WORD      TIM2_ADTR
      000000CFH   SFRSYM    DATA     BYTE      MD_DB3
      000000AFH   SFRSYM    DATA     BYTE      TIM2_ARRH
      000000A7H   SFRSYM    DATA     BYTE      TIM3_ARRH
      00000097H   SFRSYM    DATA     BYTE      TIM4_ARRH
      0000008FH   SFRSYM    DATA     BYTE      TIM5_ARRH
      000000AEH   SFRSYM    DATA     BYTE      TIM2_ARRL
      000000A6H   SFRSYM    DATA     BYTE      TIM3_ARRL
      00000087H   SFRSYM    DATA     BYTE      PCON
      000000E2H   SFRSYM    DATA     WORD      SV_US
      00000096H   SFRSYM    DATA     BYTE      TIM4_ARRL
      0000008EH   SFRSYM    DATA     BYTE      TIM5_ARRL
      000000B2H   SFRSYM    DATA     WORD      TIM2_CMTR
      00000088H   SFRSYM    DATA     BYTE      TCON
      000000AAH   SFRSYM    DATA     WORD      TIM2_CNTR
      000000A2H   SFRSYM    DATA     WORD      TIM3_CNTR
      00000092H   SFRSYM    DATA     WORD      TIM4_CNTR
      0000008AH   SFRSYM    DATA     WORD      TIM5_CNTR
      000000E5H   SFRSYM    DATA     BYTE      SV_ANGLEH
      00000086H   SFRSYM    DATA     BYTE      CFGKEY
      000000D8H   SFRSYM    DATA     BIT       PUART0
      000000E4H   SFRSYM    DATA     BYTE      SV_ANGLEL
      000000C6H   SFRSYM    DATA     WORD      MD_DAH
      000000D8H.1 SFRSYM    DATA     BIT       PUART1
      000000D8H.2 SFRSYM    DATA     BIT       PI2C0
      00000088H.2 SFRSYM    DATA     BIT       IF0
      000000CEH   SFRSYM    DATA     WORD      MD_DBH
      000000D8H.3 SFRSYM    DATA     BIT       PI2C1
      000000F0H   SFRSYM    DATA     BYTE      B
      000000C4H   SFRSYM    DATA     WORD      MD_DAL
      000000A1H   SFRSYM    DATA     BYTE      TIM2_CR0
      000000CCH   SFRSYM    DATA     WORD      MD_DBL
LX51 LINKER/LOCATER V4.66.1.0                                                         07/21/2017  11:34:04  PAGE 18


      0000009CH   SFRSYM    DATA     BYTE      TIM3_CR0
      000000A9H   SFRSYM    DATA     BYTE      TIM2_CR1
      0000009EH   SFRSYM    DATA     BYTE      TIM4_CR0
      0000009DH   SFRSYM    DATA     BYTE      TIM3_CR1
      00000089H   SFRSYM    DATA     BYTE      TIM5_CR0
      0000009FH   SFRSYM    DATA     BYTE      TIM4_CR1
      000000F8H   SFRSYM    DATA     BYTE      DRV_OUT
      00000091H   SFRSYM    DATA     BYTE      TIM5_CR1
      000000E0H   SFRSYM    DATA     BYTE      ACC
      000000F7H   SFRSYM    DATA     BYTE      PI_UKMINH
      000000C3H   SFRSYM    DATA     BYTE      MD_MAH
      000000A8H.4 SFRSYM    DATA     BIT       ES0
      000000DBH   SFRSYM    DATA     BYTE      LVSR
      000000CBH   SFRSYM    DATA     BYTE      MD_MBH
      000000C0H.4 SFRSYM    DATA     BIT       PADC0
      000000B8H   SFRSYM    DATA     BYTE      IP0
      000000F5H   SFRSYM    DATA     BYTE      PI_UKMAXH
      000000C0H.5 SFRSYM    DATA     BIT       PADC1
      000000C0H   SFRSYM    DATA     BYTE      IP1
      000000C8H   SFRSYM    DATA     BYTE      IP2
      000000F6H   SFRSYM    DATA     BYTE      PI_UKMINL
      000000C2H   SFRSYM    DATA     BYTE      MD_MAL
      00000098H.2 SFRSYM    DATA     BIT       RB8
      000000D8H   SFRSYM    DATA     BYTE      IP3
      000000CAH   SFRSYM    DATA     BYTE      MD_MBL
      000000A8H   SFRSYM    DATA     BIT       EX0
      000000F4H   SFRSYM    DATA     BYTE      PI_UKMAXL
      00000098H.3 SFRSYM    DATA     BIT       TB8
      000000B7H   SFRSYM    DATA     BYTE      TIM0_CCR1H
      000000A8H.2 SFRSYM    DATA     BIT       EX1
      000000BBH   SFRSYM    DATA     BYTE      TIM0_CCR2H
      000000D0H   SFRSYM    DATA     BIT       P
      000000BDH   SFRSYM    DATA     BYTE      TIM0_CCR3H
      000000BFH   SFRSYM    DATA     BYTE      TIM0_CCR4H
      000000C8H.2 SFRSYM    DATA     BIT       PTIM230
      000000EBH   SFRSYM    DATA     BYTE      PI_EKH
      00000098H.5 SFRSYM    DATA     BIT       SM2
      000000B6H   SFRSYM    DATA     BYTE      TIM0_CCR1L
      000000B1H   SFRSYM    DATA     BYTE      TIM0_SR1
      000000C8H.3 SFRSYM    DATA     BIT       PTIM231
      000000BAH   SFRSYM    DATA     BYTE      TIM0_CCR2L
      000000BCH   SFRSYM    DATA     BYTE      TIM0_CCR3L
      000000BEH   SFRSYM    DATA     BYTE      TIM0_CCR4L
      000000D8H.6 SFRSYM    DATA     BIT       PMCD0
      000000C8H.4 SFRSYM    DATA     BIT       PTIM450
      000000D0H.3 SFRSYM    DATA     BIT       RS0
      000000DDH   SFRSYM    DATA     BYTE      LPF_KH
      000000F3H   SFRSYM    DATA     BYTE      PI_KIH
      000000EAH   SFRSYM    DATA     BYTE      PI_EKL
      000000E8H   SFRSYM    DATA     BYTE      FOC_SET0
      000000D8H.7 SFRSYM    DATA     BIT       PMCD1
      000000C8H.5 SFRSYM    DATA     BIT       PTIM451
      000000D0H.4 SFRSYM    DATA     BIT       RS1
      000000E9H   SFRSYM    DATA     BYTE      FOC_SET1
      000000B8H.6 SFRSYM    DATA     BIT       PFOC0
      000000DCH   SFRSYM    DATA     BYTE      LPF_KL
      000000F2H   SFRSYM    DATA     BYTE      PI_KIL
      000000B8H.7 SFRSYM    DATA     BIT       PFOC1
      000000ADH   SFRSYM    DATA     BYTE      TIM2_DRH
      000000B9H   SFRSYM    DATA     BYTE      TIM0_IER
      00000083H   SFRSYM    DATA     BYTE      DPH
      000000EFH   SFRSYM    DATA     BYTE      PI_KPH
      000000A5H   SFRSYM    DATA     BYTE      TIM3_DRH
      00000095H   SFRSYM    DATA     BYTE      TIM4_DRH
      0000008DH   SFRSYM    DATA     BYTE      TIM5_DRH
LX51 LINKER/LOCATER V4.66.1.0                                                         07/21/2017  11:34:04  PAGE 19


      000000ACH   SFRSYM    DATA     BYTE      TIM2_DRL
      00000082H   SFRSYM    DATA     BYTE      DPL
      000000EEH   SFRSYM    DATA     BYTE      PI_KPL
      000000A4H   SFRSYM    DATA     BYTE      TIM3_DRL
      000000F8H.7 SFRSYM    DATA     BIT       MOE
      000000C0H.6 SFRSYM    DATA     BIT       PCMP0
      000000EDH   SFRSYM    DATA     BYTE      PI_UKH
      00000094H   SFRSYM    DATA     BYTE      TIM4_DRL
      000000C0H.7 SFRSYM    DATA     BIT       PCMP1
      000000DFH   SFRSYM    DATA     BYTE      LPF_XH
      0000008CH   SFRSYM    DATA     BYTE      TIM5_DRL
      000000AEH   SFRSYM    DATA     WORD      TIM2_ARR
      000000A8H.5 SFRSYM    DATA     BIT       MCDIE
      000000C9H   SFRSYM    DATA     BYTE      RSTSRC
      000000E7H   SFRSYM    DATA     BYTE      LPF_YH
      000000A6H   SFRSYM    DATA     WORD      TIM3_ARR
      00000088H.6 SFRSYM    DATA     BIT       MCDIF
      00000098H.4 SFRSYM    DATA     BIT       REN
      00000096H   SFRSYM    DATA     WORD      TIM4_ARR
      000000ECH   SFRSYM    DATA     BYTE      PI_UKL
      000000D7H   SFRSYM    DATA     BYTE      CMP_SR
      0000008EH   SFRSYM    DATA     WORD      TIM5_ARR
      000000DEH   SFRSYM    DATA     BYTE      LPF_XL
      000000B8H   SFRSYM    DATA     BIT       PLVD0
      000000E6H   SFRSYM    DATA     BYTE      LPF_YL
      000000B8H.1 SFRSYM    DATA     BIT       PLVD1
      000000C8H   SFRSYM    DATA     BIT       PRTC0
      000000C8H.1 SFRSYM    DATA     BIT       PRTC1
      000000E8H.7 SFRSYM    DATA     BIT       FOCEN
      000000C8H.6 SFRSYM    DATA     BIT       PTSD0
      000000D8H.4 SFRSYM    DATA     BIT       PSPI0
      000000C8H.7 SFRSYM    DATA     BIT       PTSD1
      000000D8H.5 SFRSYM    DATA     BIT       PSPI1
      0000009BH   SFRSYM    DATA     BYTE      UT_BAUDH
      000000E4H   SFRSYM    DATA     WORD      SV_ANGLE
      000000B5H   SFRSYM    DATA     BYTE      TIM2_ADTRH
      0000009AH   SFRSYM    DATA     BYTE      UT_BAUDL
      000000FCH   SFRSYM    DATA     BYTE      P0_OE
      000000FDH   SFRSYM    DATA     BYTE      P1_OE
      000000D0H.5 SFRSYM    DATA     BIT       F0
      000000B4H   SFRSYM    DATA     BYTE      TIM2_ADTRL
      000000FEH   SFRSYM    DATA     BYTE      P2_OE
      000000D0H.1 SFRSYM    DATA     BIT       F1
      00000080H   SFRSYM    DATA     BIT       GP00
      000000FFH   SFRSYM    DATA     BYTE      P3_OE
      00000090H   SFRSYM    DATA     BIT       GP10
      00000080H.1 SFRSYM    DATA     BIT       GP01
      000000A8H.6 SFRSYM    DATA     BIT       RTCIE
      000000A0H   SFRSYM    DATA     BIT       GP20
      00000090H.1 SFRSYM    DATA     BIT       GP11
      00000080H.2 SFRSYM    DATA     BIT       GP02
      000000E3H   SFRSYM    DATA     BYTE      SV_USH
      000000B0H   SFRSYM    DATA     BIT       GP30
      000000A0H.1 SFRSYM    DATA     BIT       GP21
      00000090H.2 SFRSYM    DATA     BIT       GP12
      00000080H.3 SFRSYM    DATA     BIT       GP03
      000000A8H.1 SFRSYM    DATA     BIT       TSDIE
      000000D0H   SFRSYM    DATA     BYTE      PSW
      000000B0H.1 SFRSYM    DATA     BIT       GP31
      000000A0H.2 SFRSYM    DATA     BIT       GP22
      00000090H.3 SFRSYM    DATA     BIT       GP13
      00000080H.4 SFRSYM    DATA     BIT       GP04
      000000A8H.3 SFRSYM    DATA     BIT       SPIIE
      00000088H.5 SFRSYM    DATA     BIT       TSDIF
      000000B0H.2 SFRSYM    DATA     BIT       GP32
LX51 LINKER/LOCATER V4.66.1.0                                                         07/21/2017  11:34:04  PAGE 20


      000000A0H.3 SFRSYM    DATA     BIT       GP23
      00000090H.4 SFRSYM    DATA     BIT       GP14
      00000080H.5 SFRSYM    DATA     BIT       GP05
      00000084H   SFRSYM    DATA     BYTE      FLKEY
      000000B3H   SFRSYM    DATA     BYTE      TIM2_CMTRH
      000000B0H.3 SFRSYM    DATA     BIT       GP33
      000000A0H.4 SFRSYM    DATA     BIT       GP24
      00000090H.5 SFRSYM    DATA     BIT       GP15
      00000080H.6 SFRSYM    DATA     BIT       GP06
      00000088H   SFRSYM    DATA     BIT       IT00

      01000121H   BLOCK     CODE     ---       LVL=0
      01000121H   LINE      CODE     ---       #21
      01000121H   LINE      CODE     ---       #22
      01000121H   LINE      CODE     ---       #30
      01000125H   LINE      CODE     ---       #40
      0100012CH   LINE      CODE     ---       #41
      01000130H   LINE      CODE     ---       #48
      01000136H   LINE      CODE     ---       #57
      0100013AH   LINE      CODE     ---       #63
      0100013CH   LINE      CODE     ---       #69
      0100013EH   LINE      CODE     ---       #72
      01000140H   LINE      CODE     ---       #73
      01000142H   LINE      CODE     ---       #76
      01000144H   LINE      CODE     ---       #77
      ---         BLOCKEND  ---      ---       LVL=0

      0100005BH   BLOCK     CODE     ---       LVL=0
      00000007H   SYMBOL    DATA     BYTE      Data
      0100005BH   LINE      CODE     ---       #87
      0100005BH   LINE      CODE     ---       #88
      0100005BH   LINE      CODE     ---       #89
      0100005DH   LINE      CODE     ---       #91
      01000060H   LINE      CODE     ---       #92
      01000062H   LINE      CODE     ---       #93
      ---         BLOCKEND  ---      ---       LVL=0

      ---         MODULE    ---      ---       ?C_STARTUP
      01000000H   PUBLIC    CODE     ---       ?C_STARTUP

      ---         MODULE    ---      ---       ?C?CLDPTR
      010000F2H   PUBLIC    CODE     ---       ?C?CLDPTR

      ---         MODULE    ---      ---       ?C?ILDIX
      0100010BH   PUBLIC    CODE     ---       ?C?ILDIX

      ---         MODULE    ---      ---       ?C_INIT
      010000ADH   PUBLIC    CODE     ---       ?C_START

Program Size: data=9.0 xdata=1 const=0 code=332
LX51 RUN COMPLETE.  0 WARNING(S),  0 ERROR(S)
